:0200000480007A
:100000006F000005732F2034930F80006308FF03F7
:10001000930F90006304FF03930FB0006300FF038E
:10002000130F000063040F0067000F00732F2034CC
:1000300063540F006F00400093E19153171F0000BD
:1000400023223FFC171F000023200FFC6FF01FFF2F
:100050009300000013010000930100001302000050
:100060009302000013030000930300001304000038
:100070009304000013050000930500001306000020
:100080009306000013070000930700001308000008
:10009000930800001309000093090000130A0000F0
:1000A000930A0000130B0000930B0000130C0000D8
:1000B000930C0000130D0000930D0000130E0000C0
:1000C000930E0000130F0000930F0000732540F102
:1000D0006310050097020000938202017390523072
:1000E000735044749702000093820201739052305F
:1000F00073500018970200009382020273905230EE
:10010000B70200809382F2FF7390023B9302F001EA
:100110007390023A7350403097020000938242017C
:100120007390523073502030735030309301000080
:1001300097020000938242ED739052301305100035
:100140001315F501634C05000F00F00F930110002B
:100150009308D0051305000073000000930200000F
:10016000638A020073905210B7B20000938292101B
:100170007390223073500030970200009382420146
:1001800073901234732540F17300203093012000E6
:10019000930040011301600033E720029303200025
:1001A0006314770C930130009300C0FE13016000CC
:1001B00033E720029303E0FF6318770A93014000BE
:1001C000930040011301A0FF33E7200293032000B6
:1001D000631C7708930150009300C0FE1301A0FF39
:1001E00033E720029303E0FF631077089301600078
:1001F000B70000801301100033E7200293030000D2
:100200006314770693017000B70000801301F0FFBC
:1002100033E7200293030000631877049301800002
:10022000B70000801301000033E72002B70300800D
:10023000631C7702930190009300100013010000EB
:1002400033E7200293031000631077029301A000AC
:10025000930000001301000033E720029303000025
:1002600063147700631030020F00F00F6380010009
:100270009391110093E111009308D00513850100BB
:10028000730000000F00F00F930110009308D005D9
:100290001305000073000000731000C00000000090
:1002A000000000000000000000000000000000004E
:0C02B00000000000000000000000000042
:1010000000000000000000000000000000000000E0
:1010100000000000000000000000000000000000D0
:1010200000000000000000000000000000000000C0
:1010300000000000000000000000000000000000B0
:081040000000000000000000A8
:040000058000000077
:00000001FF
